 zlib

 Timestamp is 3a07d69c (Tue Nov 07 11:17:00 2000)

 Preferred load address is 10000000

 Start         Length     Name                   Class
 0001:00000000 0000b842H .text                   CODE
 0002:00000000 0000006cH .idata$5                DATA
 0002:00000070 00001148H .rdata                  DATA
 0002:000011b8 00000028H .idata$2                DATA
 0002:000011e0 00000014H .idata$3                DATA
 0002:000011f4 0000006cH .idata$4                DATA
 0002:00001260 00000124H .idata$6                DATA
 0002:00001390 00000373H .edata                  DATA
 0003:00000000 00000004H .CRT$XCA                DATA
 0003:00000004 00000004H .CRT$XCZ                DATA
 0003:00000008 00000004H .CRT$XIA                DATA
 0003:0000000c 00000004H .CRT$XIZ                DATA
 0003:00000010 000014e0H .data                   DATA
 0003:000014f0 00000024H .bss                    DATA

  Address         Publics by Value              Rva+Base     Lib:Object

 0001:00000000       _adler32                   10001000 f   adler32.obj
 0001:00000280       _compress2                 10001280 f   compress.obj
 0001:00000349       _compress                  10001349 f   compress.obj
 0001:00000370       _get_crc_table             10001370 f   crc32.obj
 0001:0000037a       _crc32                     1000137a f   crc32.obj
 0001:00000560       _gzopen                    10001560 f   gzio.obj
 0001:00000933       _gzdopen                   10001933 f   gzio.obj
 0001:00000971       _gzsetparams               10001971 f   gzio.obj
 0001:00000dc1       _gzread                    10001dc1 f   gzio.obj
 0001:000010d4       _gzgetc                    100020d4 f   gzio.obj
 0001:0000110d       _gzgets                    1000210d f   gzio.obj
 0001:0000118f       _gzwrite                   1000218f f   gzio.obj
 0001:0000126a       _gzprintf                  1000226a f   gzio.obj
 0001:000012dc       _gzputc                    100022dc f   gzio.obj
 0001:0000131a       _gzputs                    1000231a f   gzio.obj
 0001:0000133c       _gzflush                   1000233c f   gzio.obj
 0001:000014c9       _gzseek                    100024c9 f   gzio.obj
 0001:000016d9       _gzrewind                  100026d9 f   gzio.obj
 0001:0000177d       _gztell                    1000277d f   gzio.obj
 0001:00001792       _gzeof                     10002792 f   gzio.obj
 0001:00001840       _gzclose                   10002840 f   gzio.obj
 0001:00001908       _gzerror                   10002908 f   gzio.obj
 0001:00001a30       _uncompress                10002a30 f   uncompr.obj
 0001:00001b00       _deflateInit_              10002b00 f   deflate.obj
 0001:00001b25       _deflateInit2_             10002b25 f   deflate.obj
 0001:00001e11       _deflateSetDictionary      10002e11 f   deflate.obj
 0001:00001fb1       _deflateReset              10002fb1 f   deflate.obj
 0001:00002082       _deflateParams             10003082 f   deflate.obj
 0001:0000219e       _deflate                   1000319e f   deflate.obj
 0001:00002635       _deflateEnd                10003635 f   deflate.obj
 0001:00002746       _deflateCopy               10003746 f   deflate.obj
 0001:00003f10       __tr_init                  10004f10 f   trees.obj
 0001:00004074       __tr_stored_block          10005074 f   trees.obj
 0001:000041b3       __tr_align                 100051b3 f   trees.obj
 0001:000046a2       __tr_flush_block           100056a2 f   trees.obj
 0001:000065e4       __tr_tally                 100075e4 f   trees.obj
 0001:00007310       _zlibVersion               10008310 f   zutil.obj
 0001:0000731a       _zError                    1000831a f   zutil.obj
 0001:0000732e       _zcalloc                   1000832e f   zutil.obj
 0001:00007358       _zcfree                    10008358 f   zutil.obj
 0001:00007370       _inflateReset              10008370 f   inflate.obj
 0001:000073db       _inflateEnd                100083db f   inflate.obj
 0001:00007444       _inflateInit2_             10008444 f   inflate.obj
 0001:000075aa       _inflateInit_              100085aa f   inflate.obj
 0001:000075c5       _inflate                   100085c5 f   inflate.obj
 0001:00007c96       _inflateSetDictionary      10008c96 f   inflate.obj
 0001:00007d54       _inflateSync               10008d54 f   inflate.obj
 0001:00007ea6       _inflateSyncPoint          10008ea6 f   inflate.obj
 0001:00007ee0       _inflate_blocks_reset      10008ee0 f   infblock.obj
 0001:00007f97       _inflate_blocks_new        10008f97 f   infblock.obj
 0001:0000808f       _inflate_blocks            1000908f f   infblock.obj
 0001:00009402       _inflate_blocks_free       1000a402 f   infblock.obj
 0001:0000945d       _inflate_set_dictionary    1000a45d f   infblock.obj
 0001:00009494       _inflate_blocks_sync_point 1000a494 f   infblock.obj
 0001:000094b0       _inflate_trees_bits        1000a4b0 f   inftrees.obj
 0001:00009e26       _inflate_trees_dynamic     1000ae26 f   inftrees.obj
 0001:00009fab       _inflate_trees_fixed       1000afab f   inftrees.obj
 0001:00009fe0       _inflate_codes_new         1000afe0 f   infcodes.obj
 0001:0000a035       _inflate_codes             1000b035 f   infcodes.obj
 0001:0000ad9d       _inflate_codes_free        1000bd9d f   infcodes.obj
 0001:0000adc0       _inflate_flush             1000bdc0 f   infutil.obj
 0001:0000afa0       _inflate_fast              1000bfa0 f   inffast.obj
 0001:0000b683       __CRT_INIT@12              1000c683 f   msvcrt:crtdll.obj
 0001:0000b72e       __DllMainCRTStartup@12     1000c72e f   msvcrt:crtdll.obj
 0001:0000b7cc       _strcpy                    1000c7cc f   msvcrt:MSVCRT.dll
 0001:0000b7d2       _strlen                    1000c7d2 f   msvcrt:MSVCRT.dll
 0001:0000b7d8       _memcpy                    1000c7d8 f   msvcrt:MSVCRT.dll
 0001:0000b7e0       __alloca_probe             1000c7e0 f   msvcrt:chkstk.obj
 0001:0000b7e0       __chkstk                   1000c7e0 f   msvcrt:chkstk.obj
 0001:0000b810       _memset                    1000c810 f   msvcrt:MSVCRT.dll
 0001:0000b816       _strcat                    1000c816 f   msvcrt:MSVCRT.dll
 0001:0000b81c       __initterm                 1000c81c f   msvcrt:MSVCRT.dll
 0001:0000b822       _DllMain@12                1000c822 f   msvcrt:dllmain.obj
 0002:00000000       __imp__DisableThreadLibraryCalls@4 1000d000     kernel32:KERNEL32.dll
 0002:00000004       \177KERNEL32_NULL_THUNK_DATA 1000d004     kernel32:KERNEL32.dll
 0002:00000008       __imp__fopen               1000d008     msvcrt:MSVCRT.dll
 0002:0000000c       __imp___errno              1000d00c     msvcrt:MSVCRT.dll
 0002:00000010       __imp__strcpy              1000d010     msvcrt:MSVCRT.dll
 0002:00000014       __imp___fdopen             1000d014     msvcrt:MSVCRT.dll
 0002:00000018       __imp__fprintf             1000d018     msvcrt:MSVCRT.dll
 0002:0000001c       __imp__strlen              1000d01c     msvcrt:MSVCRT.dll
 0002:00000020       __imp__sprintf             1000d020     msvcrt:MSVCRT.dll
 0002:00000024       __imp__fwrite              1000d024     msvcrt:MSVCRT.dll
 0002:00000028       __imp__fread               1000d028     msvcrt:MSVCRT.dll
 0002:0000002c       __imp__fclose              1000d02c     msvcrt:MSVCRT.dll
 0002:00000030       __imp__free                1000d030     msvcrt:MSVCRT.dll
 0002:00000034       __imp__malloc              1000d034     msvcrt:MSVCRT.dll
 0002:00000038       __imp__memcpy              1000d038     msvcrt:MSVCRT.dll
 0002:0000003c       __imp__fflush              1000d03c     msvcrt:MSVCRT.dll
 0002:00000040       __imp__fseek               1000d040     msvcrt:MSVCRT.dll
 0002:00000044       __imp__memset              1000d044     msvcrt:MSVCRT.dll
 0002:00000048       __imp__rewind              1000d048     msvcrt:MSVCRT.dll
 0002:0000004c       __imp__fputc               1000d04c     msvcrt:MSVCRT.dll
 0002:00000050       __imp__strcat              1000d050     msvcrt:MSVCRT.dll
 0002:00000054       __imp__calloc              1000d054     msvcrt:MSVCRT.dll
 0002:00000058       __imp___initterm           1000d058     msvcrt:MSVCRT.dll
 0002:0000005c       __imp___adjust_fdiv        1000d05c     msvcrt:MSVCRT.dll
 0002:00000060       __imp__ftell               1000d060     msvcrt:MSVCRT.dll
 0002:00000064       __imp__vsprintf            1000d064     msvcrt:MSVCRT.dll
 0002:00000068       \177MSVCRT_NULL_THUNK_DATA 1000d068     msvcrt:MSVCRT.dll
 0002:00000470       _deflate_copyright         1000d470     deflate.obj
 0002:00000b64       __dist_code                1000db64     trees.obj
 0002:00000d64       __length_code              1000dd64     trees.obj
 0002:00000fa0       _inflate_copyright         1000dfa0     inftrees.obj
 0002:000011b8       __IMPORT_DESCRIPTOR_MSVCRT 1000e1b8     msvcrt:MSVCRT.dll
 0002:000011cc       __IMPORT_DESCRIPTOR_KERNEL32 1000e1cc     kernel32:KERNEL32.dll
 0002:000011e0       __NULL_IMPORT_DESCRIPTOR   1000e1e0     msvcrt:MSVCRT.dll
 0003:00000000       ___xc_a                    1000f000     msvcrt:cinitexe.obj
 0003:00000004       ___xc_z                    1000f004     msvcrt:cinitexe.obj
 0003:00000008       ___xi_a                    1000f008     msvcrt:cinitexe.obj
 0003:0000000c       ___xi_z                    1000f00c     msvcrt:cinitexe.obj
 0003:000000ac       _z_errmsg                  1000f0ac     zutil.obj
 0003:00001474       _inflate_mask              10010474     infutil.obj
 0003:00001504       __adjust_fdiv              10010504     <common>
 0003:00001508       ___onexitend               10010508     <common>
 0003:0000150c       ___onexitbegin             1001050c     <common>
 0003:00001510       __pRawDllMain              10010510     <common>

 entry point at        0001:0000b72e

 Static symbols

 0001:00009558       _huft_build                1000a558 f   inftrees.obj
 0001:00003fa6       _tr_static_init            10004fa6 f   trees.obj
 0001:00003fab       _init_block                10004fab f   trees.obj
 0001:00004a5e       _build_tree                10005a5e f   trees.obj
 0001:00004dfe       _pqdownheap                10005dfe f   trees.obj
 0001:00004f9d       _gen_bitlen                10005f9d f   trees.obj
 0001:000052d0       _gen_codes                 100062d0 f   trees.obj
 0001:00005395       _build_bl_tree             10006395 f   trees.obj
 0001:0000544c       _scan_tree                 1000644c f   trees.obj
 0001:000055e9       _send_all_trees            100065e9 f   trees.obj
 0001:00005b0c       _send_tree                 10006b0c f   trees.obj
 0001:00006712       _compress_block            10007712 f   trees.obj
 0001:00006f5a       _set_data_type             10007f5a f   trees.obj
 0001:0000700c       _bi_reverse                1000800c f   trees.obj
 0001:0000704d       _bi_flush                  1000804d f   trees.obj
 0001:00007136       _bi_windup                 10008136 f   trees.obj
 0001:000071f2       _copy_block                100081f2 f   trees.obj
 0001:00002520       _putShortMSB               10003520 f   deflate.obj
 0001:00002570       _flush_pending             10003570 f   deflate.obj
 0001:00002992       _lm_init                   10003992 f   deflate.obj
 0001:00002a80       _deflate_stored            10003a80 f   deflate.obj
 0001:00002cc0       _fill_window               10003cc0 f   deflate.obj
 0001:00002efb       _read_buf                  10003efb f   deflate.obj
 0001:00002f93       _deflate_fast              10003f93 f   deflate.obj
 0001:000034ea       _longest_match             100044ea f   deflate.obj
 0001:00003819       _deflate_slow              10004819 f   deflate.obj
 0001:00000577       _gz_open                   10001577 f   gzio.obj
 0001:000009fa       _check_header              100019fa f   gzio.obj
 0001:00000bf2       _get_byte                  10001bf2 f   gzio.obj
 0001:00000ca6       _destroy                   10001ca6 f   gzio.obj
 0001:00001398       _do_flush                  10002398 f   gzio.obj
 0001:000017c9       _getLong                   100027c9 f   gzio.obj
 0001:000018c6       _putLong                   100028c6 f   gzio.obj
